S01A000064656D6F70726F675F73746D3332663734362E737265638E
S3150800800000000520E99E0008399F0008399F0008EE
S31508008010399F0008399F0008399F000800000000B2
S31508008020000000000000000000000000399F000862
S31508008030399F000800000000399F0008719F00085A
S31508008040399F0008399F0008399F0008399F0008A2
S31508008050399F0008399F0008399F0008399F000892
S31508008060399F0008399F0008399F0008399F000882
S31508008070399F0008399F0008399F0008399F000872
S31508008080399F0008399F0008399F0008399F000862
S31508008090399F0008399F0008399F0008399F000852
S315080080A0399F0008399F0008399F0008399F000842
S315080080B0399F0008399F0008399F0008399F000832
S315080080C0399F0008399F0008399F0008399F000822
S315080080D0399F0008399F0008399F0008399F000812
S315080080E0399F0008399F0008399F0008399F000802
S315080080F0399F0008399F0008399F0008399F0008F2
S31508008100399F0008399F0008399F0008399F0008E1
S31508008110399F0008399F0008399F0008399F0008D1
S31508008120399F0008399F0008399F0008399F0008C1
S31508008130399F0008399F0008399F0008399F0008B1
S31508008140399F0008399F0008399F0008399F0008A1
S31508008150399F0008399F0008399F0008399F000891
S31508008160399F0008399F0008399F0008399F000881
S31508008170399F0008399F0008399F00080000000051
S31508008180399F0008399F0008399F0008399F000861
S31508008190399F0008399F0008399F0008399F000851
S315080081A0399F0008399F0008399F0008399F000841
S315080081B0399F0008399F0008399F0008399F000831
S311080081C0399F0008399F0008EE11AA55E7
S315080081CC10B5054C237833B9044B13B10448AFF3F7
S315080081DC00800123237010BD0C0000200000000055
S315080081ECD49F000808B5034B1BB103490348AFF3EA
S315080081FC008008BD0000000010000020D49F000875
S3150800820C53B94AB9002908BF00281CBF4FF0FF31E3
S3150800821C4FF0FF3000F07AB9ADF1080C6DE904CED9
S3150800822C00F006F8DDF804E0DDE9022304B0704737
S3150800823C2DE9F0478C460D460446089E002B51D175
S3150800824C8A4217466DD9B2FA82FEBEF1000F0BD0E0
S3150800825CCEF1200C01FA0EF520FA0CFC02FA0EF7F8
S3150800826C4CEA050C00FA0EF44FEA174A250CBCFB2F
S3150800827CFAF81FFA87F90AFB18CC45EA0C4508FBED
S3150800828C09F3AB420AD9ED1908F1FF3280F02381C4
S3150800829CAB4240F22081A8F102083D44ED1AA4B283
S315080082ACB5FBFAF00AFB105544EA054400FB09F93C
S315080082BCA14509D9E41900F1FF3380F00A81A145DB
S315080082CC40F2078102383C44A4EB090440EA084012
S315080082DC0021002E61D024FA0EF40023346073605A
S315080082ECBDE8F0878B4207D9002E54D0002186E8CA
S315080082FC21000846BDE8F087B3FA83F1002940F05F
S3150800830C8E80AB4202D3824200F2FA80841A65EB65
S3150800831C03050120AC46002E3FD086E81010BDE8B8
S3150800832CF08712B90127B7FBF2F7B7FA87FEBEF149
S3150800833C000F34D1EB1B3A0C1FFA87FC0121B3FB57
S3150800834CF2F8250C02FB183345EA03450CFB08F337
S3150800835CAB4207D9ED1908F1FF3002D2AB4200F255
S3150800836CD1808046ED1AA3B2B5FBF2F002FB10558C
S3150800837C43EA05440CFB00FCA44507D9E41900F1B3
S3150800838CFF3302D2A44500F2B8801846A4EB0C04BD
S3150800839C40EA08409DE731463046BDE8F087CEF105
S315080083AC200405FA0EF307FA0EF720FA04F83A0C2D
S315080083BC25FA04F448EA0308B4FBF2F14FEA184527
S315080083CC02FB11441FFA87FC45EA044501FB0CF332
S315080083DCAB4200FA0EF409D9ED1901F1FF3080F021
S315080083EC8A80AB4240F2878002393D44EB1A1FFA69
S315080083FC88F5B3FBF2F002FB103345EA034500FBA4
S3150800840C0CF3AB4207D9ED1900F1FF386FD2AB422A
S3150800841C6DD902383D44EB1A40EA01418FE7C1F1A8
S3150800842C200722FA07F88B4005FA01F448EA0303F9
S3150800843C20FA07FE4FEA134CFD404EEA040EB5FB34
S3150800844CFCF94FEA1E440CFB19551FFA83F844EA4B
S3150800845C054509FB08F4AC4202FA01F200FA01FAE6
S3150800846C08D9ED1809F1FF3043D2AC4241D9A9F12C
S3150800847C02091D442D1B1FFA8EFEB5FBFCF00CFBE6
S3150800848C10554EEA054400FB08F8A04507D9E41830
S3150800849C00F1FF3529D2A04527D902381C4440EAF9
S315080084AC0940A4EB0804A0FB02894C45C6464D4678
S315080084BC15D312D056B1BAEB0E0364EB050404FAC5
S315080084CC07F7CB401F43CC40376074600021BDE8EA
S315080084DCF0871846F8E69046E0E6C245EAD2B8EBCD
S315080084EC020E69EB03050138E4E72846D7E7404650
S315080084FC91E78146BEE7014678E702383C4445E7F2
S3150800850C084608E7A8F102083D442BE7704700BF68
S3150800851C08B50948094B03604FF4614343600023CF
S3150800852C8360C36003610C2242618361C361036289
S3150800853C436201F070FB08BD500000200048004063
S3150800854C2DE9F04104460D461746984601F03EF8CB
S3150800855C154BA3FB00308009002201E00132D2B290
S3150800856C112A1ED8114B13F8121003EB420393F879
S3150800857C01E001EB0E0303FB0443B0FBF3FC03FB26
S3150800858C1C06002EEAD11FFA8CF32B80013B9BB2FA
S3150800859CB3F5806FE2D2397088F800E00120BDE8A7
S315080085ACF0810020BDE8F081D34D6210EC9F0008E5
S315080085BC70B58CB00025ADF82E508DF82D500CAB3F
S315080085CC03F8045D0DF12D020DF12E014FF4FA702E
S315080085DCFFF7B6FF1A4C1B4B236025766576A576F6
S315080085EC0126E67625776577A560E5609DF82D303A
S315080085FC013B1B0423619DF82C30013B1B05636171
S3150800860CBDF82E306360204600F02FF906950795C5
S3150800861C08964CF6E043019302954FF6E0730393E4
S3150800862C04230493059509960E230A9301A920465B
S3150800863C00F0C2F9204600F055FA0CB070BD00BF28
S3150800864C280000200064004008B5002301220146DA
S3150800865C034801F031FA08B1002008BD012008BD15
S3150800866C5000002008B5FFF753FFFFF7A1FF08BD20
S3150800867CBFF34F8F0549CA6802F4E062044B1343F3
S3150800868CCB60BFF34F8F00BFFDE700BF00ED00E0E6
S3150800869C0400FA0508B5214B1B78B3B92048FFF737
S315080086ACD3FF012800D008BD1D4B1B78013BDBB25C
S315080086BC3F2BF8D801F052FC1A4B18600122174BC5
S315080086CC1A700022184B1A7008BD174B1B78013309
S315080086DC13481844FFF7B8FF01280AD001F03EFCEE
S315080086EC104B1B6864339842DDD900220B4B1A7069
S315080086FCD9E70D4A13780133DBB21370084A12789E
S3150800870C9342D0D10021054A1170054A5278FF2AA6
S3150800871CC9D1022BC7D1FFF7ABFF00BF110100204F
S3150800872CD0000020140100201201002000B58BB0E7
S3150800873C01AB03AA00210E4800F002FA30B940F248
S3150800874C6763039A9A4204D0002343B90BB05DF8C9
S3150800875C04FB059B0BB10023F7E70123F5E79DF80E
S3150800876C0430FF2BF2D1079B022BEFD1FFF780FFCA
S3150800877C2800002008B5FFF78DFFFFF7D7FF08BDC7
S3150800878C08B500228021024800F0D0FB08BD00BFC6
S3150800879C0004024010B501F0E1FB0E4B1B68C31A2E
S315080087ACB3F5FA7F0CD304460B4B1B784BB9012255
S315080087BC094B1A708021094800F0B8FB054B1C6060
S315080087CC10BD0022044B1A708021044800F0AEFB41
S315080087DCF4E700BF1C010020180100200004024029
S315080087EC10B504460E4B18784FF47A73B3FBF0F3B6
S315080087FC0C4A1068B0FBF3F000F07EFA68B90F2C3F
S3150800880C01D9012010BD002221464FF0FF3000F09F
S3150800881C43FA054B1C60002010BD012010BD00BF9B
S3150800882C00000020080000200400002008B50320E2
S3150800883C00F020FA0020FFF7D3FF01F0B9FA002068
S3150800884C08BD0000034A1168034B1B780B441360E0
S3150800885C704700BF2001002000000020014B18685B
S3150800886C704700BF200100207047002800F0A18047
S3150800887C38B5044690F82030D3B12268136823F033
S3150800888C02031360FFF7EAFF054623685A6812F0DD
S3150800889C020F10D0FFF7E2FF401B0A28F5D9636ACE
S315080088AC43F400336362052384F82030012038BD75
S315080088BCFFF7DAFFE1E71A6842F001021A60FFF7E0
S315080088CCCDFF054623685A6812F0010F0DD1FFF744
S315080088DCC5FF401B0A28F5D9636A43F40033636263
S315080088EC052384F82030012038BD227E012A3DD08C
S315080088FC1A6822F080021A60637E012B3BD022682C
S3150800890C136823F040031360A37E012B39D0226829
S3150800891C136823F020031360E37E012B37D02268FB
S3150800892C136843F010031360237F012B35D022689C
S3150800893C136823F008031360637F012B33D0226876
S3150800894C136823F0040313602168A368E2681343D1
S3150800895C22691343626913436268013A1343CB6174
S3150800896C00206062012384F8203038BD1A6842F072
S3150800897C80021A60C0E72268136843F0400313604C
S3150800898CC2E72268136843F020031360C4E7226821
S3150800899C136823F010031360C6E72268136843F0C4
S315080089AC08031360C8E72268136843F004031360CE
S315080089BCCAE701207047000090F82030013BDBB273
S315080089CC012B05D9436A43F480234362012070477F
S315080089DC70B4434BD3F8002242F00102C3F80022CC
S315080089ECD3F8002222F47C52C3F80022D3F80022D2
S315080089FC486A42EA0022C3F800224A6902F01F02BA
S31508008A0C012000FA02F2D3F81C42D0430440C3F802
S31508008A1C1C42CB69B3B9324BD3F80C420440C3F8A9
S31508008A2C0C424C69CE688D8845EA0645483443F8AD
S31508008A3C34504D698E680C8844EA0644483503EB75
S31508008A4CC5035C60CB69012B1DD08B69002B32D119
S31508008A5C234CD4F804320340C4F804320B698BBB9C
S31508008A6C1F4BD3F814422040C3F814020B6A012B8F
S31508008A7C2FD01B4AD2F8003223F00103C2F8003279
S31508008A8C002070BC7047164BD3F80C421443C3F83D
S31508008A9C0C424C690E688D8845EA0645483443F8FD
S31508008AAC34504D698E688C8944EA0644483503EB84
S31508008ABCC5035C60C9E70A4CD4F804321343C4F8FE
S31508008ACC0432CBE70648D0F814321343C0F81432F4
S31508008ADCCCE7034BD3F81C120A43C3F81C22C8E78D
S31508008AEC0064004038B590F82030DBB2012B05D075
S31508008AFC436A43F400234362012038BD044602232B
S31508008B0C80F820300268136823F001031360FFF71E
S31508008B1CA5FE054623685B6813F0010F0DD0FFF719
S31508008B2C9DFE401B0A28F5D9636A43F40033636239
S31508008B3C052384F82030012038BD0020606238BD3A
S31508008B4C30B490F82040013CE4B2012C06D9436AB3
S31508008B5C43F480234362012030BC704700296FD14F
S31508008B6C0468E46814F0030F64D0056801F11B046B
S31508008B7C24012C5904F004049460002C6BD105686C
S31508008B8C01F11B0424012C59640D1460056801F1CC
S31508008B9C1B0424012D59C5F34005D56005682544E9
S31508008BAC6D6805F00F051561056825446D68C5F3F4
S31508008BBC0725956105682C446468240C546104687F
S31508008BCC0A011444D4F8B8411C7004681444D4F847
S31508008BDCB841C4F307245C7004681444D4F8B8414B
S31508008BECC4F307449C7004681444D4F8B841240EA2
S31508008BFCDC7004681444D4F8BC411C710468144431
S31508008C0CD4F8BC41C4F307245C7104681444D4F842
S31508008C1CBC41C4F307449C7104682244D2F8BC21B5
S31508008C2C120EDA71F9B90268D36843F02003D360DF
S31508008C3C002091E7436A43F40013436201208BE753
S31508008C4C0468246914F0030F8FD1436A43F40013A4
S31508008C5C4362012080E7056801F11B0424012C59A5
S31508008C6CE408546092E70268136943F02003136121
S31508008C7C002071E70649CB6823F4E0631B041B0C40
S31508008C8C000200F4E0600343024A1A43CA607047C4
S31508008C9C00ED00E00000FA0530B4144BDB68C3F3B2
S31508008CAC0223C3F10704042C28BF04241D1D062D1A
S31508008CBC13D9033B012505FA04F4013C21409940DC
S31508008CCC05FA03F3013B13401943002807DB090196
S31508008CDCC9B2074B195430BC70470023EAE700F0B9
S31508008CEC0F000901C9B2034B1954F4E700ED00E073
S31508008CFC00E400E014ED00E00138B0F1807F0AD200
S31508008D0C064B5860F021064A82F82310002098601A
S31508008D1C07221A6070470120704700BF10E000E078
S31508008D2C00ED00E0042805D0054A136823F0040377
S31508008D3C13607047024A136843F0040313607047C4
S31508008D4C10E000E0704708B5FFF7FCFF08BD00000F
S31508008D5CF0B583B0002437E0092600E0002606FAB1
S31508008D6C0EF6324302336C4E46F823206B4B1A68C8
S31508008D7CEB4302EA03064F6817F4803F01D045EA35
S31508008D8C0206664A1660526803EA02064F6817F42A
S31508008D9C003F01D045EA0206604A5660926803EA2B
S31508008DAC02064F6817F4801F01D045EA02065B4A93
S31508008DBC9660D26813404E6816F4001F01D045EA37
S31508008DCC0203564AD36001340F2C00F2A380012308
S31508008DDCA3400A6803EA0205AB42F4D14A68122A90
S31508008DEC18BF022A12D14FEAD40E0EF1080E50F80B
S31508008DFC2E2004F00706B6000F27B74022EA070212
S31508008E0C0F6907FA06F6324340F82E2006684FEA31
S31508008E1C440E032202FA0EF2D24316404F6807F0AC
S31508008E2C030707FA0EF73E4306604E68771E112EA7
S31508008E3C18BF012F01D9122E0FD186681640CF689C
S31508008E4C07FA0EF73E438660466826EA03034E6821
S31508008E5CC6F30016A64033434360C3681A408B68B2
S31508008E6C03FA0EF31A43C2604B6813F0805FAAD05C
S31508008E7C2B4B5A6C42F480425A645B6C03F4804365
S31508008E8C0193019BA3089E1C234A52F8262004F042
S31508008E9C03064FEA860E0F2606FA0EF622EA060295
S31508008EAC204FB8423FF45AAF1F4EB04222D006F5B7
S31508008EBC8066B04220D006F58066B0421ED006F514
S31508008ECC8066B0421CD006F58066B0421AD006F50C
S31508008EDC8066B04218D006F58066B04216D006F504
S31508008EEC8066B04214D006F58066B0423FF434AFC3
S31508008EFC0A2634E7012632E7022630E703262EE750
S31508008F0C04262CE705262AE7062628E7072626E759
S31508008F1C082624E703B0F0BD00380140003C0140A8
S31508008F2C00380240000002400004024012B909044D
S31508008F3C816170478161704710B582B01B4B1A6C02
S31508008F4C42F080521A641B6C03F080530193019B08
S31508008F5C174A136843F480331360FFF77FFC044603
S31508008F6C134B5B6813F4803F08D1FFF777FC001BA3
S31508008F7CB0F57A7FF4D9032002B010BD0C4A1368F9
S31508008F8C43F400331360FFF769FC0446084B5B682F
S31508008F9C13F4003F07D1FFF761FC001BB0F57A7F8D
S31508008FACF4D90320E8E70020E6E700BF00380240C2
S31508008FBC00700040002800F0DB8170B582B00446D2
S31508008FCC036813F0010F3AD0A24B9B6803F00C030D
S31508008FDC042B2BD09F4B9B6803F00C03082B20D03B
S31508008FEC6368B3F5803F50D0002B54D1994B1A685F
S31508008FFC22F480321A601A6822F480221A60636896
S3150800900C002B5FD0FFF72AFC0546924B1B6813F41E
S3150800901C003F14D1FFF722FC401B6428F5D9032026
S3150800902CABE18C4B5B6813F4800FD9D0894B1B686A
S3150800903C13F4003F03D06368002B00F09B81236870
S3150800904C13F0020F64D0834B9B6813F00C0F4DD0B2
S3150800905C804B9B6803F00C03082B42D0E368002B6B
S3150800906C79D07C4A136843F001031360FFF7F6FBCB
S3150800907C0546784B1B6813F0020F63D1FFF7EEFB1E
S3150800908C401B0228F5D9032077E1724A136843F48A
S3150800909C80331360B3E7B3F5A02F09D06D4B1A686C
S315080090AC22F480321A601A6822F480221A60A6E723
S315080090BC684B1A6842F480221A601A6842F48032A5
S315080090CC1A609CE7FFF7CAFB0546624B1B6813F44C
S315080090DC003FB4D0FFF7C2FB401B6428F5D9032028
S315080090EC4BE15C4B5B6813F4800FB7D1594B1B688B
S315080090FC13F0020F04D0E368012B01D001203CE1E8
S3150800910C544A136823F0F803216943EAC103136030
S3150800911C236813F0080F46D0636983B34D4A536F1F
S3150800912C43F001035367FFF799FB0546494B5B6F01
S3150800913C13F0020F37D1FFF791FB401B0228F5D924
S3150800914C03201AE1434A136823F0F803216943EA1A
S3150800915CC1031360DCE73F4A136823F0010313606D
S3150800916CFFF77CFB05463B4B1B6813F0020FCFD071
S3150800917CFFF774FB401B0228F5D90320FDE0354A9E
S3150800918C536F23F001035367FFF768FB0546314B12
S3150800919C5B6F13F0020F06D0FFF760FB401B02282B
S315080091ACF5D90320E9E0236813F0040F7ED0294B88
S315080091BC1B6C13F0805F31D1264B1A6C42F080522F
S315080091CC1A641B6C03F080530193019B0125224BF7
S315080091DC1B6813F4807F23D0A368012B34D0002B93
S315080091EC3CD11C4B1A6F22F001021A671A6F22F037
S315080091FC04021A67A368002B46D0FFF72FFB064616
S3150800920C144B1B6F13F0020F4FD1FFF727FB801B74
S3150800921C41F288339842F3D90320AEE00025D6E70D
S3150800922C0D4A136843F480731360FFF717FB064661
S3150800923C094B1B6813F4807FCED1FFF70FFB801BFD
S3150800924C6428F5D9032098E0024A136F43F001030A
S3150800925C1367CFE70038024000700040052B09D091
S3150800926C484B1A6F22F001021A671A6F22F0040291
S3150800927C1A67BFE7434B1A6F42F004021A671A6F54
S3150800928C42F001021A67B5E7FFF7E8FA06463D4BC6
S3150800929C1B6F13F0020F08D0FFF7E0FA801B41F2A0
S315080092AC88339842F3D9032067E0F5B9A369002BF4
S315080092BC62D0344A926802F00C02082A5FD0022B5C
S315080092CC19D0304A136823F080731360FFF7C6FA77
S315080092DC04462C4B1B6813F0007F47D0FFF7BEFAE9
S315080092EC001B0228F5D9032047E0264A136C23F005
S315080092FC80531364DAE7234A136823F080731360E8
S3150800930CFFF7ACFA05461F4B1B6813F0007F06D017
S3150800931CFFF7A4FA401B0228F5D903202DE0E369D0
S3150800932C226A1343626A43EA8213A26A5208013A12
S3150800933C43EA0243E26A43EA026343F00053114AE2
S3150800934C5360136843F080731360FFF787FA04467B
S3150800935C0C4B1B6813F0007F06D1FFF77FFA001B36
S3150800936C0228F5D9032008E0002006E0002004E0D6
S3150800937C01207047012000E0002002B070BD0120DA
S3150800938CFBE700BF00380240F8B5314B9B6803F089
S3150800939C0C03042B59D0082B01D02E48F8BD2C4BA6
S315080093AC5A6802F03F025B6813F4800F2AD0284BE8
S315080093BC5B68C3F388131E4600275C010025E41A74
S315080093CC65EB0705A90141EA9461A001001B61EB55
S315080093DC0501CB0043EA5073C400A01943EB0701FF
S315080093EC4B0243EAD0534402204619460023FEF7A3
S315080093FC07FF174B5B68C3F3014301335B00B0FBF4
S3150800940CF3F0F8BD124B5B68C3F388131E460027AE
S3150800941C5C010025E41A65EB0705A90141EA94618C
S3150800942CA001001B61EB0501CB0043EA5073C40095
S3150800943CA01943EB07018B0243EA9053840220469A
S3150800944C19460023FEF7DCFED3E70348F8BD00BF38
S3150800945C003802400024F40000127A00002800F0BC
S3150800946CA28070B50446524B1B6803F00F038B425F
S3150800947C0CD24F4A136823F00F030B43136013687F
S3150800948C03F00F03994201D0012070BD236813F035
S3150800949C020F17D013F0040F04D0464A936843F40E
S315080094ACE0539360236813F0080F04D0414A93687D
S315080094BC43F4604393603F4A936823F0F003A06833
S315080094CC034393600D46236813F0010F31D063688C
S315080094DC012B20D0022B25D0364A126812F0020F27
S315080094EC63D034498A6822F0030213438B60FFF772
S315080094FCB5F906462F4B9B6803F00C036268B3EB71
S3150800950C820F16D0FFF7AAF9801B41F288339842CE
S3150800951CF0D9032070BD274A126812F4003FE0D137
S3150800952C012070BD234A126812F0007FD9D10120A0
S3150800953C70BD1F4B1B6803F00F039D420CD21C4ACF
S3150800954C136823F00F032B431360136803F00F0300
S3150800955C9D4201D0012070BD236813F0040F06D07C
S3150800956C144A936823F4E053E1680B439360236829
S3150800957C13F0080F07D00F4A936823F46043216948
S3150800958C43EAC1039360FFF7FFFE0A4B9B68C3F3DC
S3150800959C0313094AD35CD840084B18600020FFF720
S315080095AC1FF9002070BD01207047012070BD00BF57
S315080095BC003C02400038024010A0000808000020B9
S315080095CC014B1868704700BF0800002008B5FFF764
S315080095DCF7FF044B9B68C3F38223034AD35CD8403A
S315080095EC08BD00BF0038024020A0000808B5FFF7E8
S315080095FCE7FF044B9B68C3F34233034AD35CD8405A
S3150800960C08BD00BF0038024020A0000870470000C3
S3150800961C10B5044683680269134342691343C26949
S3150800962C1343016808689C4A024013430B6022687E
S3150800963C536823F44053E1680B435360A369226AC9
S3150800964C134321688A6822F4306213438B602368BB
S3150800965C924A93422BD0924A93423BD0914A9342D8
S3150800966C50D0914A934263D0904A934275D0904A0F
S3150800967C934200F08A808F4A934200F09E808E4A6D
S3150800968C934200F0B2801023E269B2F5004F00F065
S3150800969CD480082B00F26F81DFE813F03201470102
S315080096AC51016D015A016D016D016D016401834B08
S315080096BCD3F8903003F00303032B09D8DFE803F043
S315080096CC0204AD060123DFE70423DDE70823DBE705
S315080096DC1023D9E7794BD3F8903003F00C030C2BF5
S315080096EC0ED8DFE803F0070D0D0D090D0D0D9C0DB9
S315080096FC0D0D0B000023C7E70423C5E70823C3E7B2
S3150800970C1023C1E76D4BD3F8903003F03003102BC0
S3150800971C0AD006D9202B00F08480302B06D10823DA
S3150800972CB2E71BB90023AFE70423ADE71023ABE779
S3150800973C624BD3F8903003F0C003402B09D005D9FF
S3150800974C802B70D0C02B06D108239DE71BB90023AC
S3150800975C9AE7042398E7102396E7584BD3F89030EA
S3150800976C03F44073B3F5807F0BD007D9B3F5007FAC
S3150800977C5BD0B3F5407F06D1082385E71BB90023D8
S3150800978C82E7042380E710237EE74C4BD3F890300E
S3150800979C03F44063B3F5806F0BD007D9B3F5006FAC
S315080097AC45D0B3F5406F06D108236DE71BB90123E5
S315080097BC6AE7042368E7102366E7404BD3F8903032
S315080097CC03F44053B3F5805F0BD007D9B3F5005FAC
S315080097DC2FD0B3F5405F06D1082355E71BB90023F4
S315080097EC52E7042350E710234EE7344BD3F8903056
S315080097FC03F44043B3F5804F0BD007D9B3F5004FAC
S3150800980C19D0B3F5404F06D108233DE71BB9002301
S3150800981C3AE7042338E7102336E7022334E7022312
S3150800982C32E7022330E702232EE702232CE7022332
S3150800983C2AE7022328E7022326E7082B5DD8DFE868
S3150800984C03F0051F3F5C485C5C5C5300FFF7BEFEEB
S3150800985C6268530803EB4003B3FBF2F39BB2002098
S3150800986CA3F110014FF6EF72914200F287809AB27B
S3150800987C22F00F02C3F3420313432268D36050E06D
S3150800988CFFF7B4FE6268530803EB4003B3FBF2F32D
S3150800989C9BB20020E4E700BFF369FFEF001001401C
S315080098AC0044004000480040004C00400050004076
S315080098BC0014014000780040007C0040003802404B
S315080098CC6268304B03EB5203B3FBF2F39BB20020F6
S315080098DCC6E7FFF759FD6268530803EB4003B3FB71
S315080098ECF2F39BB20020BBE76268530803F580339A
S315080098FCB3FBF2F39BB20020B2E701200023AFE7DB
S3150800990CFFF764FE626800EB5203B3FBF2F39BB2FB
S3150800991C0020A3F110014FF6EF72914230D822685D
S3150800992CD36000232366636610BDFFF75FFE62688B
S3150800993C00EB5203B3FBF2F39BB20020E9E7626833
S3150800994C114B03EB5203B3FBF2F39BB20020E0E797
S3150800995CFFF71AFD626800EB5203B3FBF2F39BB2F6
S3150800996C0020D6E76268530803F50043B3FBF2F30D
S3150800997C9BB20020CDE701200023CAE70120D0E7DF
S3150800998C0120CEE70048E8010024F400436A13F0EE
S3150800999C010F06D00268536823F40033816A0B431F
S315080099AC5360436A13F0020F06D00268536823F417
S315080099BC8033C16A0B435360436A13F0040F06D015
S315080099CC0268536823F48023016B0B435360436A84
S315080099DC13F0080F06D00268536823F40043416B52
S315080099EC0B435360436A13F0100F06D00268936852
S315080099FC23F48053816B0B439360436A13F0200F57
S31508009A0C06D00268936823F40053C16B0B4393602A
S31508009A1C436A13F0400F0AD00268536823F4801384
S31508009A2C016C0B435360036CB3F5801F0BD0436A70
S31508009A3C13F0800F06D00268536823F40023816C58
S31508009A4C0B43536070470268536823F4C003416C98
S31508009A5C0B435360EBE72DE9F04105460F461646D6
S31508009A6C9846069C2B68DB6937EA03030CBF01236F
S31508009A7C0023B3421DD1B4F1FF3FF3D0FEF7EEFE3F
S31508009A8CA0EB0800844201D3002CEBD12A6813689A
S31508009A9C23F4D07313602A68936823F00103936048
S31508009AAC20236B67AB67002385F870300320BDE86D
S31508009ABCF0810020BDE8F0812DE9F04383B01E4605
S31508009ACC836F202B03D0022003B0BDE8F083044635
S31508009ADC0D469046002A18BF002976D090F87030AB
S31508009AEC012B01D10220EFE7012380F87030002307
S31508009AFCC36722238367FEF7B1FE0746A4F858808E
S31508009B0CA4F85A80A368B3F5805F06D0A3B9226976
S31508009B1C72B9FF22A4F85C2014E0226922B940F23B
S31508009B2CFF12A4F85C200DE0FF22A4F85C2009E0E3
S31508009B3C7F22A4F85C2005E0B3F1805F0AD00022EE
S31508009B4CA4F85C20B4F85C80B3F5805F0CD04FF0B9
S31508009B5C00091EE022691AB97F22A4F85C20F1E7F5
S31508009B6C3F22A4F85C20EDE7236913B14FF00009F6
S31508009B7C0FE0A94600250CE023685B6A08EA030394
S31508009B8C29F8023BB4F85A309BB2013B9BB2A4F8B5
S31508009B9C5A30B4F85A309BB28BB100963B46002229
S31508009BAC20212046FFF757FF88B9002DE4D02368FB
S31508009BBC5A6A5FFA88F3134005F8013BE2E720235B
S31508009BCCA367002084F870007EE701207CE7032059
S31508009BDC7AE710B582B004460023C367FEF73EFE4B
S31508009BEC2268126812F0080F07D120236367A3674F
S31508009BFC002084F8700002B010BD6FF07E4300930D
S31508009C0C034600224FF400112046FFF724FF0028D4
S31508009C1CEBD00320EFE768B310B50446436F03B3E4
S31508009C2C242363672268136823F001031360204614
S31508009C3CFFF7EEFC01281FD0636ABBB9226853688C
S31508009C4C23F4904353602268936823F02A039360A5
S31508009C5C2268136843F0010313602046FFF7B9FF27
S31508009C6C10BD80F87030FFF7D1FCD9E72046FFF716
S31508009C7C8DFEE3E70120704710BD000010B40F4AB3
S31508009C8CD2F8883043F47003C2F888300C4B196844
S31508009C9C41F001011960002098601C6809492140AF
S31508009CAC196009495960196821F480211960D8602E
S31508009CBC4FF0006393605DF8044B704700ED00E0CD
S31508009CCC00380240FFFFF6FE10300024014B024A12
S31508009CDC9A60704700ED00E00080000800B595B06A
S31508009CEC3022002108A800F067F900230393049397
S31508009CFC059306930793214B1A6C42F080521A640B
S31508009D0C1B6C03F080530193019B1D4B1A6842F49C
S31508009D1C40421A601B6803F440430293029B0123DA
S31508009D2C08934FF4A023099302230E934FF4800251
S31508009D3C0F92082210924FF4D87211921293139321
S31508009D4C08A8FFF737F900B1FEE7FFF7F5F800B1F9
S31508009D5CFEE70F23039302230493002305934FF482
S31508009D6CA05306934FF480530793072103A8FFF7D4
S31508009D7C75FB00B1FEE715B05DF804FB0038024030
S31508009D8C0070004008B5FFF7A1FFFEF74FFDFFF77F
S31508009D9CA5FF00F0CDF8FEF7F3FC08BD08B5FFF7F4
S31508009DACF1FFFEF75FFCFEF7F5FCFEF7E3FCFAE7BE
S31508009DBC2DE9F0418CB0464B1A6C42F080521A646D
S31508009DCC1A6C02F080520192019A5A6C42F4804243
S31508009DDC5A645A6C02F480420292029A1A6B42F046
S31508009DEC02021A631A6B02F002020392039A1A6BA6
S31508009DFC42F008021A631A6B02F008020492049ADB
S31508009E0C1A6C42F480221A641A6C02F480220592A7
S31508009E1C059A1A6C42F000721A641B6C03F00073F4
S31508009E2C0693069B0320FEF725FF002211466FF0CA
S31508009E3C0B00FEF731FF002211466FF00A00FEF701
S31508009E4C2BFF002211466FF00900FEF725FF0022B2
S31508009E5C11466FF00400FEF71FFF002211466FF043
S31508009E6C0300FEF719FF002211466FF00100FEF7FA
S31508009E7C13FF002211464FF0FF30FEF70DFF80232B
S31508009E8C079301230893002409940A94114D07A9F2
S31508009E9C2846FEF75DFF4FF44078CDF81C80022764
S31508009EAC0897099403260A9607230B9307A90A48C9
S31508009EBCFEF74EFFCDF81C80089709940A960923DD
S31508009ECC0B9307A92846FEF743FF0CB0BDE8F081B3
S31508009EDC0038024000040240000C0240DFF834D07F
S31508009EEC002103E00C4B5B58435004310B480C4BD8
S31508009EFC42189A42F6D30B4A02E0002342F8043B76
S31508009F0C094B9A42F9D3FFF7B9FE00F031F8FFF77F
S31508009F1C45FF70470000052038A000080000002007
S31508009F2C0C0000200C00002024010020FEE7000095
S31508009F3C08B5FFF745FB084BA3FB00308009FEF775
S31508009F4CDBFE0420FEF7EEFE002211464FF0FF3032
S31508009F5CFEF7A2FE08BD00BFD34D621008B5FEF78A
S31508009F6C7DFC08BD08B5FEF76DFCFEF7ECFE08BDDA
S31508009F7C70B50D4E0D4CA41BA4100025A54209D195
S31508009F8C0B4E0C4C00F020F8A41BA4100025A5427F
S31508009F9C05D170BD56F8253098470135EEE756F8C9
S31508009FAC253098470135F2E730A0000830A00008A4
S31508009FBC30A0000834A0000802440346934200D19E
S31508009FCC704703F8011BF9E7F8B500BFF8BC08BCE5
S31508009FDC9E467047F8B500BFF8BC08BC9E4670474D
S31508009FEC05020602060307030803090309040A0403
S31508009FFC0B040C040C050D050E050F050F061006B3
S3150800A00C10071008000000000000000001020304FD
S3110800A01C06070809000000000102030402
S30D0800A02814E2FF7F01000000AD
S3090800A030F1810008A4
S3090800A034CD810008C4
S3110800A03801000000100000000024F400E5
S70508009EE96B
